:10000000830100308A002228F20003088301B60031
:1000100083120313A20B0E28A20A0F2885140B11BA
:10002000FF30AA07031CAB032B082A04031D1C285E
:10003000C430AA00AB012015851036088300F20EEB
:10004000720E09002030840021302F2021308400DE
:1000500034302F208301172E04068001840A040601
:10006000031D2C280034B400B51B3D2835088A0038
:100070003408B40A0319B50A8200831335188317AC
:100080003408B40A84000008080041346E3479341E
:1000900020346B3465347934203474346F34203434
:1000A00072346534743472347934003441346E34CB
:1000B000793420346B3465347934203474346F34BB
:1000C0002034733474346134723474340034323410
:1000D000303430343234203442346F34623420349B
:1000E00042346C34693463346B34003450346F34CC
:1000F00077346534723420346F34663466340034B7
:10010000723465346D346F34743465346D346934ED
:10011000643469342034763430342E34333400344B
:1001200042346F346F34743420346634613469344B
:100130006C34653464342E34003442346F346F349C
:10014000743469346E34673420344C3449344E345A
:10015000553458342E342E342E34003482070E3465
:10016000113417341934173411340E340034023476
:1001700006340E341E340E3406340234003408348F
:100180000C340E340F340E340C340834003408347C
:1001900008340834003400340034003400340034AF
:1001A0000E341F341F341F340E34003400348207E1
:1001B0000334033402340234013482074C345234A1
:1001C000553444342E3482076C34723475346434BC
:0201D0002E34CB
:1009700083120313AF009500080083120313B00025
:10098000803E342D01303425CD30B200B301092D25
:1009900083120313B1008316981CCC2C83123108E8
:1009A00099000800831203139818D82C181DDA2C0C
:1009B000181218161A080800831203139501043040
:1009C0009200FF30831692000F30831297000800C8
:1009D00040303425AF0100308A002F08AE201E259C
:1009E000AF0A28302F0203180800EB2CFF2C300828
:1009F000B5002F08AF0A0319B00A33201E25831251
:100A000003133008B5002F083320003803190800FD
:100A1000F72C831203131010F001F1013208700259
:100A2000B2003308031C330A7102B3008F0032088E
:100A30008E0010140C100C1808001B2D83120313C9
:100A4000B10005150F3086053108F039860406140B
:100A500006100F308605310EF03986040614061094
:100A60000630B200B3010B2D83120313B100051140
:100A70000F3086053108F0398604061406100F3051
:100A80008605310EF0398604061406100630B200D1
:100A9000B3010B2D83120313B2011030B1000530E6
:100AA000AF005F2D0F308605310886040A30B00094
:100AB000B00B582D0518612DB20A0310B10DAF0B04
:100AC000522D320808008312031386013130831639
:100AD000850006308600073083129F00C430AA00CC
:100AE000AB0120110A30A4000230A6000430A5009A
:100AF000A010A201A20A1430A800AC01AD01A90106
:100B000001308316990022309800903083129800AB
:100B1000831681128B168B173130831290000800D8
:100B20008312031305116A30B2001830B30009258F
:100B30000F30860530308604061406107130B2007E
:100B40000230B3000925061406100F30B200B301BD
:100B50000925061406107130B2000230B3000925D1
:100B60000F308605861606140610B200B30109255B
:100B700028303425083034250C3034250630342D07
:100B800083120313AF00A01CDD2DA010D02D2F0861
:100B9000BD2C2F08A10008002F08342D2F081E2D72
:100BA0002708013A0319C72D113A0319C92D023A32
:100BB0000319CC2D063A0319CE2D20302F02031C29
:100BC000F12D0B2E1030342DC22C1430342DA201F7
:100BD00008001030342520301E251030342D003010
:100BE000BD2C2F08023A0319E22D013A0319E42D16
:100BF000053A0319E52D013A0319E72D0F3A0319B8
:100C0000E92D023A0319EF2D073A0319EF2DA0142D
:100C10002F08A700080080302F02031C152EA030DB
:100C20002F020318152E0730AF052F081E2D632540
:100C3000DC242430B200F430B30009259025C2240E
:100C4000FF30A100B8248030AF000030B000F6249F
:100C5000E8244030BD2400301E256730AF0000304E
:100C6000B000F6242430B200F430B3000925A2010C
:100C70002430B200F430B30009250030B8248C1EB3
:100C8000C42ED224C0252014C42E851ED72EA90A16
:100C90008515C2249D30AF000030B000F6248430AA
:100CA000AC000330AD000830A30020102012D72E76
:100CB000201C662E2010A30300302D022D300319B6
:100CC0002C020318662E2D30AC00AD01A3080319C9
:100CD000A90A2D082C04031D7D2E0530A9008511BD
:100CE000C2249030AF000030B000F6244030BD2464
:100CF0004530AF000030B000F624051ED72E201678
:100D0000D72E201C872E20102D30AC00AD01851E63
:100D1000A01D8C2E5A30C824201A051A912EAC0121
:100D2000AD012D082C04031DD72E8511C224763069
:100D3000AF000030B000F6240730AC00AD01851ED6
:100D4000AB2E0430A9004030BD245630AF00003037
:100D5000B000F624D72E0330B82E2D082C04031D26
:100D6000D72EA901D72E2D082C04031DD72E053010
:100D7000A900D72E851ED72E4A25AE00043A0319A6
:100D8000D72EA901C224D72E2908F0000630700200
:100D90000318D72E06308A00D130700703188A0A4C
:100DA0008200452E582E812EAD2EB32EBA2EA01DB8
:100DB000E82EA0112D082C040319E22EAC0803190B
:100DC000AD03AC03851EE62E2108E72E0030B824C3
:100DD000201D3F2E20114A25F326A80B3F2E14304C
:100DE000A800A0153F2E83120313AF00043A031D81
:100DF000012F2508043A031DFF2EB001EC2F02300D
:100E00000E2F2508043A031D0A2FB001B00A2F083F
:100E1000A500EC2FA4080319102F0330B000EC2F0D
:100E200004300E2F0A30A400A601A60A08000030E4
:100E30008A002508DD20C824A20108000A30A40089
:100E4000A601A60A0430A5000800A408031DA403F7
:100E50000800A60B080000308A002508DD20C82401
:100E60000230A60008003008F000053070020318B8
:100E7000080007308A004030700703188A0A820091
:100E8000122F172F1E2F252F292F0A30A400A6015D
:100E9000A60A080000308A002508DD20C824A20127
:100EA000080000308A002508E320C8240A30A40086
:100EB000A601A60A0430A500A20108003008F0002F
:100EC000053070020318080007308A006B30700785
:100ED00003188A0A8200452F4A2F512F0800080064
:100EE000952F0A30A400A601A60A0800A408031939
:100EF0007F2F00308A002508DD20C824A2010A3097
:100F0000A400A601A60A0430A5000800A408031D39
:100F1000A4030800A60803190800A60100308A00EF
:100F20002508E320C824A20108003008F00005309D
:100F300070020318080007308A00A23070070318F7
:100F40008A0A8200712F0800762F862F8A2F0A3096
:100F5000A400A601A60A08000A30A6000800A408FA
:100F60000319B82F00308A002508DD20C824A2010B
:100F70000A30A400A601A60A0430A5000800A408AF
:100F8000031DA403080026080A3A031DCD2F0030D4
:100F90008A002508E320C824A201A60B080000301F
:100FA0008A002508E320C8240230A6000800300883
:100FB000F000053070020318080007308A00E430A2
:100FC000700703188A0A8200A72FAC2FAF2FBF2FFC
:100FD000C32F0430A500080000308A002508D72060
:100FE000F000043070020318E92F07308A00FC304B
:100FF000700703188A0A8200332F5E2F952FD72F90
:02400E00013D72
:00000001FF
